:100000000C94A4060C94DC060C94DC060C94DC0620
:100010000C94DC060C94DC060C94DC060C94DC06D8
:100020000C94DC060C94DC060C948A1E0C94CC1DFB
:100030000C94C3240C94DC060C94DC060C94DC06B3
:100040000C94DC060C94DC060C94DC060C94DC06A8
:100050000C94DC060C9476240C94DC060C94DC06E0
:100060000C94DC060C94DC060C94DC060C94DC0688
:100070000C94DC060C94DC060C94DC060C94DC0678
:100080000C94DC060C94DC060C94DC060C94DC0668
:100090000C94DC060C94DC060C94DC060C94DC0658
:1000A0000C94DC060C94DC060C94DC06070C0A0CA1
:1000B000350C550C5B0C660C690C690C690C8A0DCF
:1000C0008A0DDC0CDE0CE30C070D280D2B0D2E0D1C
:1000D000510D700D7B0D5D10D11065102F10331078
:1000E000691036106C1077104110C71045107B1046
:1000F00049107F10A9104D108310B31053108910B0
:1001000093103A1070103D10731058108E109F10FD
:10011000BF10C1102B106110DA1003110911F41077
:10012000FA100F1115111B11C511C511F811F81195
:1001300076129C139C139C13941208131913191311
:10014000E513011406140B14101415141A141F14BB
:10015000241429142E14351438143B143E1441145D
:10016000441447144A144F14E40FE41B0B1CB41D31
:100170000B1CB41D571C7A1CB41D6F1D7F1D00DAAB
:100180000281FFD9F1DB20A4A62EAF00A0C000A100
:10019000C800AED580A81FD300408D1420000004F5
:1001A0007F3F1F643214643214783C1E1E140A050B
:1001B0008D8E8F9091ADAEAFB0B1CDCECFD0D100FE
:1001C00088898A8B8CA8A9AAABACC8C9CACBCC0039
:1001D0008384858687A3A4A5A6A7C3C4C5C6C70074
:1001E000000000000000000000000000000000000F
:1001F00000000000000000000000000000000000FF
:10020000000000007E0F00D4FFFFFFC70000007851
:1002100000000000000000002A2B28000000000061
:1002200000000000000000000000002900000000A5
:100230002C1E3420212224342627252E362D373813
:10024000271E1F202122232425263333362E37381C
:100250001F0405060708090A0B0C0D0E0F101112DA
:10026000131415161718191A1B1C1D2F3130232DA6
:10027000350405060708090A0B0C0D0E0F101112A4
:10028000131415161718191A1B1C1D2F3130354C55
:1002900005010980A101850319012AB7001501266E
:1002A000B700950175108100C0050C0901A10185F9
:1002B0000419012AA002150126A0029501751081DA
:1002C00000C00660FF0961A1010962150026FF0058
:1002D0009520750881020963150026FF0095207599
:1002E000089102C005010906A101050719E029E7E7
:1002F0001500250195087501810295017508810198
:100300000507190029FF150026FF009506750881CD
:1003100000050819012905950575019102950175DA
:10032000039101C009025B00030100A0FA09040067
:100330000001030101000921110100012240000711
:1003400005810308000109040100020300000009FF
:10035000211101000122220007058203200001076C
:100360000503032000010904020001030000000945
:10037000211101000122320007058403200001122F
:1003800001000200000008504401000001010200C9
:100390000112034B0069006E007400730075006762
:1003A0000069000000140341004400500065006E25
:1003B0000072006F00730065000000040309040070
:1003C00000000000003E5B4F5B3E003E6B4F6B3E0B
:1003D000001C3E7C3E1C00183C7E3C18001C577DD7
:1003E000571C001C5E7F5E1C0000183C180000FFBC
:1003F000E7C3E7FF00001824180000FFE7DBE7FF72
:100400000030483A060E00262979292600407F054B
:10041000050700407F05253F005A3CE73C5A007F16
:100420003E1C1C0800081C1C3E7F0014227F221466
:10043000005F5F005F5F0006097F017F0000668943
:10044000956A0060606060600094A2FFA29400085A
:10045000047E04080010207E20100008082A1C08D2
:1004600000081C2A0808001E10101010000C1E0C9A
:100470001E0C0030383E383000060E3E0E060000DE
:10048000000000000000005F0000000007000700FF
:1004900000147F147F1400242A7F2A1200231308DB
:1004A000646200364956205000000807030000002F
:1004B0001C224100000041221C00002A1C7F1C2A33
:1004C0000008083E08080000807030000008080896
:1004D0000808000000606000002010080402003ED0
:1004E0005149453E0000427F40000072494949465B
:1004F000002141494D33001814127F100027454553
:100500004539003C4A49493100412111090700366B
:100510004949493600464949291E00000014000097
:10052000000040340000000008142241001414149C
:100530001414000041221408000201590906003E6B
:10054000415D594E007C1211127C007F49494936A9
:10055000003E41414122007F4141413E007F4949E7
:100560004941007F09090901003E41415173007F63
:100570000808087F0000417F4100002040413F0102
:10058000007F08142241007F40404040007F021C51
:10059000027F007F0408107F003E4141413E007F02
:1005A00009090906003E4151215E007F09192946CB
:1005B0000026494949320003017F0103003F4040C2
:1005C000403F001F2040201F003F4038403F006355
:1005D00014081463000304780403006159494D436F
:1005E00000007F4141410002040810200000414109
:1005F000417F0004020102040040404040400000EE
:1006000003070800002054547840007F28444438F1
:1006100000384444442800384444287F0038545467
:1006200054180000087E09020018A4A49C78007FDA
:10063000080404780000447D4000002040403D0054
:10064000007F102844000000417F4000007C0478B7
:100650000478007C08040478003844444438007C62
:100660001824241800182424187C007C080404088A
:100670000048545454240004043F4424003C4040A7
:10068000207C001C2040201C003C4030403C0044AA
:1006900028102844004C9090907C004464544C44B2
:1006A00000000836410000000077000000004136DD
:1006B0000800000201020402003C2623263C000040
:1006C000000000000000000000000000000000002A
:1006D0000000000000000080C0C0E0F0F0F8FCBCAA
:1006E0009E9EBCFCF8F0F0E0C0C08000000000005E
:1006F000000080C0F0FCFE8EE67000FCFEFEFC00F8
:100700003878F0FEFEF078380000000000000000AD
:1007100000787878787878787E7EFEFCFC7C18000B
:100720009EBC1C020F1E0C00000000000000000018
:1007300000000000000000000000000000E0F0F0F9
:10074000F0E0ECEEF7F37020007C7C7C7E007E7E97
:100750007E7F7F7F000080C0E07E5B4F5BFEC0003D
:1007600000C000DCD7DEDEDED7DC00C00000000009
:100770000000000000000000000000000000000079
:100780000000000000000000000000000000000069
:1007900000000000000001E1E1E1E1E3E7E7E3E35D
:1007A000FFFFE3E3E7E7E3E1E1E1E101000000004F
:1007B000000040F1FBFFFFE7F3F800FFFFFFFF87BA
:1007C000C7E7FFFFFFFFE7C7870700000000000043
:1007D000008E9E9E1E1E1E1E1E1E9FDFFFFFFECF52
:1007E0000F0F0700000000000000000000000000E4
:1007F000000000000000000000000000000F1F3F8C
:100800007F7F7F7F7F3F1E0C001F1F1F3F003F3FEA
:100810003F7F7F7F00307B7F7830202030787F3BA8
:100820000003000F7F0F0F0F7F0F00030000000079
:1008300000000000000000000000000000000000B8
:1008400000000000000000000000000000000000A8
:1008500000000000000070707173737F7E7C707008
:100860007F7F70707C7E7F737371707000000000FA
:100870000000607C3E013E610E1E003F7F7F7F7363
:1008800073717077777071737373000000000000EC
:10089000001F7F7F787878787878797B7B7B03017D
:1008A0000000000000000000000000000000000048
:1008B0000000000000000000000000000000000038
:1008C0000000000000000000000000000000000028
:1008D0000000000000000000000000000000000018
:1008E0000000000000000000000000000000000008
:1008F000000000000000000000000000000000FFF9
:10090000AA7F55402223252628292A2C2D2F303234
:10091000333536383A3B3D3E4042434547494A4CE1
:100920004E5051535557595A5C5E6062646668690F
:100930006B6D6F71737577797B7D7F818385878917
:100940008A8C8E90929496989A9C9E9FA1A3A5A71C
:10095000A8AAACAEAFB1B3B4B6B8B9BBBCBEBFC148
:10096000C2C3C5C6C7C9CACBCCCDCED0D1D2D2D3D3
:10097000D4D5D6D7D7D8D9D9DADADBDBDBDCDCDCE7
:10098000DCDCDDDDDDDDDCDCDCDCDCDBDBDBDADAAA
:10099000D9D9D8D7D7D6D5D4D3D2D2D1D0CECDCC21
:1009A000CBCAC9C7C6C5C3C2C1BFBEBCBBB9B8B636
:1009B000B4B3B1AFAEACAAA8A7A5A3A19F9E9C9AC1
:1009C00098969492908E8C8A89878583817F7D7B8F
:1009D00079777573716F6D6B6968666462605E5C70
:1009E0005A5957555351504E4C4A49474543424036
:1009F0003E3D3B3A3836353332302F2D2C2A2928CC
:100A00002625232200AF00AE29001E001F00200073
:100A10002100220023002B0014001A0008001500FA
:100A200017001C00390004001600070009000A0026
:100A30000B00E1001D001B0006001900050011005D
:100A4000E000E300E2000000000000002C002400B1
:100A50002500260027002D002E002A0018000C007B
:100A6000120013002F00300031000D000E000F00A7
:100A7000330034002800A80010003600370038008A
:100A8000E500520023520000000021522252500083
:100A900051004F0001003A003B003C003D003E0089
:100AA0003F00010001000100010001000100010000
:100AB000007C0100010001000100010001000100B3
:100AC000010001000100010001000100010001001E
:100AD0000100000000000000010040004100420051
:100AE0004300440045004C000100010001000100EA
:100AF00001000100010001000100010001000100EE
:100B00000100AE0001000100010001000100010030
:100B100001000000000001000100010001000100CF
:100B200001000100010001000100010001000100BD
:100B300001000100010001000100010001000100AD
:100B4000010001000100010001000100010001009D
:100B5000010001000100010001000100010000008E
:100B6000000000000100010001000100010001007F
:100B7000010001000100010001000100010001006D
:100B80000100010001000100010001000100AB00B3
:100B9000010001000100010001000100010000004E
:100BA000000001000100010001000100010001003E
:100BB000010001000100010001000100010001002D
:100BC000010001000100010001000100010001001D
:100BD000010001000100010001000100010001000D
:100BE0000100010001000100010000000000000000
:100BF00001000100010001000100010001000100ED
:100C000001000100010001000100010001000100DC
:100C100001000100010001000100010001000100CC
:100C200001000100010001000100000000000100BE
:100C30000100010001000100A900AA00010001005B
:100C40000100010001000100000101010101010199
:100C50000101020202020202020202030303030371
:100C60000303030404040404040405050505050640
:100C700006060606070707070708080808090909FE
:100C8000090A0A0A0B0B0B0C0C0C0D0D0D0E0E0EA7
:100C90000F0F0F1010111111121213131414151538
:100CA00016161717181819191A1A1B1B1C1D1D1EAA
:100CB0001E1F2020212222232424252626272829FE
:100CC000292A2B2C2D2D2E2F30313232333435362C
:100CD0003738393A3B3C3D3E3F404142434445462C
:100CE0004748494A4C4D4E4F505153545556585908
:100CF0005A5B5D5E5F616264656668696B6C6D6FAF
:100D00007072737577787A7B7D7E80828385878821
:100D10008A8C8E8F91939596989A9C9EA0A2A3A55B
:100D2000A7A9ABADAFB1B3B5B7BABCBEC0C2C4C65C
:100D3000C9CBCDCFD1D4D6D8DBDDDFE2E4E7E9EB18
:100D4000EEF0F3F5F8FAFDFF11241FBECFEFDAE065
:100D5000DEBFCDBF04B603FE18C08091E5049091BC
:100D6000E604A091E704B091E8048730904BA740D7
:100D7000B04B59F41092E5041092E6041092E70487
:100D80001092E804E0E0F8E3099511E0A0E0B1E09A
:100D9000E0E8F8E502C005900D92A03BB107D9F755
:100DA00024E0A0EBB1E001C01D92A53EB207E1F73F
:100DB0000E94DE060C943E2C0C940000CF93DF932F
:100DC000CDB7DEB7C454D1090FB6F894DEBF0FBE5D
:100DD000CDBF85B7806885BF85B7806885BF84B77C
:100DE000877F84BF0FB6F894A895809160008861D2
:100DF00080936000109260000FBE90E080E80FB614
:100E0000F89480936100909361000FBE8AE594E1AD
:100E10009093B1018093B0010E94101E0E942F1E7A
:100E20008091E20084608093E200789480915D027A
:100E30008823A1F01091E9001F709091EC00892F98
:100E4000817090FD80E8182B1092E9008091E800F5
:100E500083FD0E94011B1F701093E90082E084BD96
:100E600093E095BD9AEF97BD80936E000E94E81FB6
:100E7000811102C00E94D81F81E08093D001279881
:100E80002F9A55985D9A8FE891E00197F1F700C08D
:100E900000004091D001E1EDF1E020E0241779F06D
:100EA00083B190E0880F892F881F990B4D9B02C05A
:100EB00032E001C030E0832B81932F5FEFCF0EE152
:100EC00011E088E2E82E81E0F82ED8018D918D01A5
:100ED0008F3F11F00E949F14E016F106B1F708E26F
:100EE00011E0BFE2EB2EB1E0FB2EF80181918F0102
:100EF0008F3F11F00E949F14E016F106B1F78AE0CF
:100F0000E5EFF1E0DF01282F1D922A95E9F7E2EBEA
:100F1000F1E0DF011D928A95E9F70E9474168111B4
:100F200002C00E94801682E090E00E945C2B8093B9
:100F3000C30184E090E00E946A2B9093BD018093EE
:100F4000BC010E945919EFE3FCE93197F1F700C0A9
:100F500000000E9459198091F50180FF08C06FEFD1
:100F60007FEF80E090E00E948E2B0E94522483E06D
:100F700090E00E945C2B0E94FC2783E08093F201AA
:100F800080E2809368020E94142A6DE070E081E99B
:100F900091E00E94DA1A892B09F043C08091F20196
:100FA00063E070E081FD3AC08EE891E00E94DA1AB9
:100FB000892BB9F56DE070E08EE791E00E94DA1AB6
:100FC000892B79F50E94AB24DC01CB0180549B4234
:100FD000AE4FBF4F8093B3049093B404A093B50475
:100FE000B093B604EBE6F2E080E092E0DF019C0112
:100FF0001D9221503040E1F7F0937204E0937104A8
:101000008FEF9FEF90936A028093690281E0809353
:10101000B8048093B7041092F30103C08BE891E009
:10102000C5CF8091BE01811133C00E947416811119
:1010300004C00E9480160E94782988E090E00E94F7
:10104000642B6093AE047093AF048093B0049093CC
:10105000B1046E7F71F40E94782988E090E00E94CC
:10106000642B6093AE047093AF048093B0049093AC
:10107000B1040E94022910927A048091AE0480FF8C
:1010800004C060E086950E94282981E08093BE011B
:1010900080E091E09093BF048093BE0422242394C7
:1010A000312CCE0101967C0180915D02853009F0E2
:1010B00067C0F0E4DF2ECC24C39400E112E18091FC
:1010C0005D02853009F04FC080915D02843009F4E3
:1010D00038C010927A048091C00181110DC0C09275
:1010E000C0018091AE04982F91709093BF018E7FC4
:1010F0008093AE040E941C200E94D7261092C20446
:10110000A8E1B0E00FB6F894A895A09360000FBED8
:10111000D092600083B7817F846083BF83B7816092
:1011200083BF7894889583B78E7F83BF0FB6F8947A
:10113000A8958091600088618093600010926000A3
:101140000FBE80915C02882309F4B9CF0E9459191F
:10115000E5EFF1E081918111E6C42FEF31E02E1728
:101160003F07C1F7ACCF0E9436280E94502510924D
:10117000C0018091BF0181110E9423230E942D2371
:101180000E945919E4ECCE2EE1E0DE2E85EF91E0CD
:1011900023969FAF8EAF2397DC01F60191918D913D
:1011A00021E0EE3CF20719F09817C1F322C0981322
:1011B00020C00E94B7248C018091C1019091C2018E
:1011C0000817190709F4C5C48FEF8DAB8EAB1FAAA2
:1011D0000E94B7248160782F99AF88AF4DA95EA98E
:1011E0006FA989AD0E94CA0D1093C2010093C1017D
:1011F000B0C475EFA72E71E0B72E10E0D5017D9039
:101200005D01F6018080872401F100E09924939428
:10121000882D8921A1F00AAF1BAF91E0872D89218C
:1012200009F490E09CAF0E94B7248160782F9EAFB4
:101230008DAF4AAD5BAD6CAD8EAD0E94CA0D0F5F38
:10124000990C073029F7D6017C921F5FBFEFCB1AAC
:10125000DB0A1A3099F60E94AB24AA24A394809149
:101260007A04882309F493C080917904E091AE0454
:10127000E695E81BE0937504823059F4F0E0E455FC
:10128000FE4FE4910E2F10E06EE4C62E62E2D62EE1
:1012900059C0863059F4F0E0E755FE4FE4910E2F27
:1012A00010E05EE3C52E52E2D52E4CC0893061F4C9
:1012B000E695F0E0EA55FE4FE4910E2F10E041EB89
:1012C000C42E41E2D42E3EC08F3061F4E695F0E0AA
:1012D000ED55FE4FE4910E2F10E033E5C32E31E2C1
:1012E000D32E30C0853159F4F0E0E056FE4FE49142
:1012F0000E2F10E025E0C22E21E2D22E23C088312D
:10130000A1F0833249F4EEE9F1E0059114919CEEED
:10131000C92E91E2D92E16C0843271F000ED17E08B
:1013200084E9C82E8FE1D82E0DC008E210E0BAE89B
:10133000CB2EB0E2DB2E06C004EF11E0A2E5CA2EF0
:10134000A0E2DA2E80917604882361F01092760470
:101350000E94B724909374048093730410927804CD
:10136000109277040E94B724E0917304F091740402
:101370008E1B9F0B8F3F9F4750F40E0F1F1F109324
:1013800074040093730483E794E0F6010995912CAB
:10139000B12CEDEF8E2E77247394FCEF5F2E8091AD
:1013A000D001981608F0A6C0092D10E083B190E096
:1013B000880F892F881F990B4D9B02C0E2E001C066
:1013C000E0E08E2BD801AF52BE4FEC912E2F237050
:1013D00030E0482F082E000C550B2417350709F470
:1013E00087C0EE0FEE0FE82BEC93EF70F0E0E15DBD
:1013F000FE4F980121533E4F69019081D9018C9194
:10140000890F8C93843094F1F801E253FE4F808170
:101410008F5F80830E94B7249BA65CA67DA6816017
:10142000782F9FA78EA7492D5CEF61E08FA50E94C2
:10143000CA0DEFE3FCE93197F1F700C000000E940C
:10144000B72498AA59AA1AAA8160782F9CAB8BABB3
:10145000492D5CEF60E08CA90E94CA0D8FE39CE9E6
:101460000197F1F700C0000021E001C020E0D601A3
:101470008C918D3F8CF5F801E253FE4F80818150B5
:1014800080830E94B72499A28AA27BA28160782FD0
:101490009DA38CA3492D5DEF61E08DA10E94CA0D33
:1014A000EFE3FCE93197F1F700C000000E94B72498
:1014B0009EA28FA218A68160782F9AA789A7492D8E
:1014C0005DEF60E08AA50E94CA0D8FE39CE9019759
:1014D000F1F700C0000021E0D6018C91082E000C2D
:1014E000990B64E070E00E94B02BF6018083B22A71
:1014F000939455CFB1100E94AB248091B8048823F7
:1015000009F42EC180E00E94BC1A83E00E94BC1A3C
:1015100080ED91E00E94AE1A87E00E94BC1A80EC38
:1015200091E00E94AE1A8BE00E94BC1A80EB91E021
:101530000E94AE1A8091690290916A02892B31F45F
:101540008091B704882309F40BC1F3C08091B804DB
:101550008823B1F38091F3018111F2CF0E94F1262B
:101560002091690230916A022115310549F380E02A
:10157000482E512C6101082E02C0CC0CDD1C0A94AF
:10158000E2F7A60142235323452B11F48F5FF0CFDE
:101590009091F201920165E0220F331F6A95E1F705
:1015A00090FF13C055E0369527955A95E1F7220F25
:1015B000220F220F20930A0110920D01295F209320
:1015C0000B0183E080930E0111C08295880F807615
:1015D00080930A01220F232F221F330B3195209372
:1015E0000D01815E80930B0110920E0124E630E024
:1015F00047E050E068E071E088E70E94BC2A892B50
:1016000009F09ECF8091F20180FF72C080E2E2ED8E
:10161000F1E0DF011D928A95E9F735E0440C551C95
:101620003A95E1F7E3E4F1E02596FFAFEEAF2597B9
:101630006FE371E02596AEADBFAD25978D912596F0
:10164000BFAFAEAF2597FB019191BF01A201490F3A
:10165000511D45595D4F90E08E529E4FFC0107E0B1
:101660009F01281B390B822C01C0880C2A95EAF7B0
:1016700021965FAF4EAF2197912C2196AEADBFADB5
:1016800021971D912196BFAFAEAF21971821202F32
:1016900029192770722E022E000C330BB12F01C0B6
:1016A000BB0F7A94EAF77B2E31952195310927708B
:1016B000332701C016952A95EAF7712A1081712AFD
:1016C0007082939428E09212D8CF015031960F3F48
:1016D00039F625968EAD9FAD25978754914009F038
:1016E000A9CF04E610E020E230E042ED51E00DC069
:1016F000C20125E0880F991F2A95E1F7AC014559F1
:101700005D4F04E610E020E230E060E488E70E94EC
:10171000DD2A892B09F014CFC094D09480916902FE
:1017200090916A02C822D922D0926A02C0926902BC
:1017300007CF0E94AB240091B3041091B404209110
:10174000B5043091B604DC01CB01801B910BA20BD8
:10175000B30B8F3F9F4FAF4FBF4710F40E94D72668
:10176000A11001C0B1100E94F1260E945025909155
:10177000F401891721F08093F4010E94AB24809139
:101780005D02843009F090CC83E08093E900809181
:10179000E80082FF89CC8091E80085FF22C00E948A
:1017A000611F81111CC000E210E09E012F5F3F4FBE
:1017B000690108C08091F100D6018D936D0101503F
:1017C000110969F08091E80085FDF4CF8091E8006F
:1017D0008B778093E8000E94611F882399F391E042
:1017E00001C090E08091E8008B778093E800992316
:1017F00009F45ACC2981822F90E0FC013197E53120
:10180000F10508F087C1EA5AFF4F0C94E62B1A82C3
:101810008BE0D7C08A81823009F49DC150F48130B9
:1018200009F078C10E94AB249B838C837D836E83F7
:1018300073C1833041F0843009F06CC11B821C827B
:101840001D821E8269C1FE013396CE010D9623963C
:10185000AEADBFAD23972D912396BFAFAEAF23970B
:101860002193E817F90799F757C18A81823019F057
:10187000853051F04FC16B817C818D819E810E94AA
:10188000EC2B0E94172748C18091AE0480FF0AC04C
:101890008091AE048E7F8093AE0410927A040E94F1
:1018A0001C203AC10E94232337C14C816B818A815D
:1018B0000E94A9261EC12D813E813227232732276F
:1018C0004C816B818A810E94372626C10E945E2648
:1018D00023C18A81823009F01DC12830B9F1293035
:1018E00009F45FC08B818230F9F098F4813009F0FF
:1018F00013C18C81BFEF8B9FC00111246FEF70E08B
:101900000E94082B462F20E06091B0048091AF0424
:101910001AC08330A1F0843009F0FEC020E040916D
:10192000B1046D818C810FC08C81882309F4B0CF04
:101930000E94232360E08C810E942829EDC08C81C5
:101940008093B204E9C00E946222E6C08B8182309B
:10195000E1F078F4813009F0DFC08091B104EFEF5D
:101960008E9FC00111246FEF70E00E94082B6C83E2
:10197000D3C0833091F0843009F0CEC08091AF04A1
:101980008C838091B0048D83C7C08091AE0480FFAA
:1019900002C0869504C080E002C08091B2048C83AE
:1019A000BBC06091AE047091AF048091B00490917F
:1019B000B1040E941529B0C080E14EC081E08A8345
:1019C0008AE98B83A9C00A811B8110270127102770
:1019D000AC80B12C6701C8018A599D4F96012E1920
:1019E0003F092A153B0508F097C00A39F1E01F07A7
:1019F00030F40E945C2BD60114968C9302C0F60141
:101A000014820F5F1F4FFFEFCF1ADF0AE4CF0A8166
:101A10001B81102701271027AC80B12C6701C8015A
:101A20008A599D4F96012E193F092A153B0508F04A
:101A300073C00A3921E0120728F4D60114966C917C
:101A40000E94702B0F5F1F4FBFEFCB1ADB0AE7CF4F
:101A50000E94C62561C084E08A835EC00A811B8122
:101A6000102701271027AC80B12C6701C80186968A
:101A700096012E193F092A153B0508F04DC0003389
:101A8000E2E01E0730F40E945C2BD60114968C9382
:101A900002C0F60114820F5F1F4FFFEFCF1ADF0A5B
:101AA000E5CF0A811B81102701271027AC80B12CBC
:101AB0006701C801869696012E193F092A153B0534
:101AC00058F5003322E0120728F4D60114966C91E1
:101AD0000E94702B0F5F1F4FBFEFCB1ADB0AE9CFBD
:101AE00041E08C81811101C040E06B818A810E94BC
:101AF00003269D8337C02D813E813227232732273D
:101B000041E08C81811101C040E06B818A810E949B
:101B1000D62502C08FEF898340E250E0B70182E012
:101B20000E94F923C1CA09BD19BD09B400FEFDCF49
:101B30008091D8008F7D8093D8008091E0008260F2
:101B40008093E0008091E00081FDFCCF0E94362868
:101B5000B6CAA12C84CB85E290E00E945C2B1B824C
:101B60001C821D828E83D8CF0E9436282FEF84E3FB
:101B70009CE0215080409040E1F700C000009CE0D4
:101B800088E10FB6F894A895809360000FBE9093FB
:101B90006000FFCFA7E1B0E0E0EDFDE00C942B2B5F
:101BA0004B8B5C8B6D8B7E8B8F8B611110924902FE
:101BB00086E09E01235F3F4FD901E82F1D92EA95F1
:101BC000E9F795E0FE017396D90101900D929A957F
:101BD000E1F79C894E895F897B897D879E876F8726
:101BE000598B488BF901DE01179601900D928A9569
:101BF000E1F7CE0107960E94D21781113EC086E020
:101C0000FE013796DE01119601900D928A95E1F75B
:101C1000FF81E8856A857B856115710531F0EF3FAD
:101C200031F481E0FF3F19F403C081E001C080E09E
:101C300080FD23C020910E0230E0C901019687701B
:101C4000992740913F0250E08417950779F1F98375
:101C5000EA837D836C8396E0929FD001939FB00DC1
:101C60001124A15FBD4FFE01319601900D929A950E
:101C7000E1F780930E020E945F1716E080913F0209
:101C800090910E028917F9F0189FC0011124815F0D
:101C90009D4F0E94D2178823B1F080913F0290E0BF
:101CA00001968770992780933F02E8CF0E943628DB
:101CB00010920E0210923F02E8E0F2E086E0DF01AF
:101CC0001D928A95E9F76796E3E00C94472BADE007
:101CD000B0E0EDE6FEE00C941C2BFC0180819181CC
:101CE00023813481232B31F09F3F31F491E08F3FEA
:101CF00019F403C091E001C090E090FDD7C57F01C9
:101D000085E0DE01199601900D928A95E1F7F701C1
:101D1000228189859A85222349F00E947127182FF4
:101D2000682F89859A850E94C62703C00E94AD2727
:101D3000182F69857A85812F0E94B6148C01F701CE
:101D40008281882309F436C1980122503747203117
:101D5000310508F04BC18FEF93E00E945C2B81119D
:101D600033C1025036E6A32E32E0B32E002379F0C1
:101D7000A114F4E0BF0609F427C1C5010E945C2B41
:101D8000811101C001502FEFA21AB20AEFCFCE018C
:101D900001962C0188E0F20111928A95E9F72AE078
:101DA000322E85010F5F1F4FC5010E945C2B898376
:101DB0001A82882309F408C1813009F041C0650105
:101DC000F2E0CF0ED11CC8010E945C2B8A838823CD
:101DD00009F4FAC09FEF980F933060F423E0A20E4D
:101DE000B11CC6010E945C2B8B83882309F4ECC0D4
:101DF0001C8229C0843031F54E0133E0830E911CE2
:101E000002E010E056018FEFA81AB80AC6010E943E
:101E10005C2BF40181934F01882309F4D5C08C37E2
:101E200041F4E2E0F0E0EC0FFD1FE00FF11F108243
:101E30000AC00F5F1F4F65010730110519F7C4C0B5
:101E4000580101C056018201F8012081222309F4C2
:101E5000A8CF213009F04CC08181813049F468015C
:101E6000F2E0CF0ED11CF80182810E94E5280AC061
:101E7000823051F46801F2E0CF0ED11CF80182816A
:101E80000E949028860189C0833049F46801F2E0FD
:101E9000CF0ED11CF80182810E945D28F3CF8430DF
:101EA00019F00F5F1F4F79C0F80122810E5F1F4F9D
:101EB00080E090E030E0205331092A30310568F4A9
:101EC000389EA001399E500D1124C901840F951F21
:101ED0000F5F1F4FF8012081EDCF009709F45DC01F
:101EE000EFE9FFE03197F1F700C000000197F5CF6F
:101EF000E22FF0E0E05FFD4F2490822F86958695DB
:101F0000869590E0FC01E050FE4F64902770712CA4
:101F1000022E02C0759467940A94E2F7F1E06F22F2
:101F20007724FC01E051FE4F8490912C022E02C0D8
:101F3000959487940A94E2F731E083229924FC0176
:101F4000E052FE4FC490D12C02C0D594C7942A957C
:101F5000E2F781E0C822DD246114710419F081EEFA
:101F60000E9490288114910419F086EE0E94902816
:101F7000822D0E94E5288114910419F086EE0E94BA
:101F80005D286114710419F081EE0E945D28C1146E
:101F9000D10419F08CE20E94E5280F5F1F4F8BE0FF
:101FA000815009F451CFEFE9FFE03197F1F700C01C
:101FB0000000F6CF011537E7130709F042C181E0B1
:101FC0000E94E3270E94CE1A80914002877009F494
:101FD0006DC4F7018281882309F468C48091BD0132
:101FE00082FF64C482E00E942B1760C40115F7E7EA
:101FF0001F0711F481E005C0013027E7120721F423
:1020000082E00E94F027DECFF801E851FC47E7307C
:10201000F10508F4E5C0882309F45BC11092BB0404
:10202000C8019057839708F013C184E090E00E94A4
:102030006A2B9093BD018093BC01F801E150F047F9
:10204000E232F10520F4E559FF4F0C94E62B809124
:10205000BC018160ACC08091BD018860B4C080913A
:10206000BC018260A4C08091BC0120C08091BC01F1
:1020700088609DC08091BD011EC08091BD018260BD
:10208000A2C08091BC01806192C08091BC0180623D
:102090008EC08091BC0180648AC00E9436288091E5
:1020A000BC01806884C08091BC01886084607FC06E
:1020B0008091BD018260816086C08091BC018E7F6D
:1020C00076C08091BD01877F7EC08091BC018D7FED
:1020D0006EC08091BC0120C08091BC01877F67C029
:1020E0008091BD011EC08091BD018D7F6CC080912B
:1020F000BC018F7E5CC08091BC018F7D58C08091F7
:10210000BC018F7B54C00E9436288091BC018F7720
:102110004EC08091BC01877F8B7F49C08091BD01FB
:102120008D7F8E7F50C08091BC0182FB222720F9D9
:1021300091E0922790FB82F990FB83F938C080915F
:10214000BD01982F909591708E7F892B90FB81F91E
:102150003AC08091BC0186FB222720F991E09227AA
:1021600090FB86F924C00E9436288091BC0187FB31
:10217000222720F991E0922790FB87F918C061E0AF
:1021800001C060E08EE090E00E94702B1EC0809144
:10219000BC0184FB222720F991E0922790FB84F96F
:1021A00006C08091BC01982F909590FB80F9809398
:1021B000BC010BC08091BD0183FB222720F991E077
:1021C000922790FB83F98093BD016091BC017091CF
:1021D000BD0184E090E00E948E2B0E943628F4CE50
:1021E000E357FF4F0C94E62B06E221EE41EE6AE145
:1021F0007CE705C007E225EE45EE6BE17CE7C70111
:102200000E945D25E1CE06E221EE40EE68E17CE72A
:10221000F6CF07E225EE44EE69E17CE7F0CF06E277
:1022200021EE42EE6CE17CE7EACF07E225EE46EED6
:102230006DE17CE7E4CF08E221E045EE6EE17CE76A
:10224000DECF013097E7190709F0DECE82E0B8CE85
:102250000631ECE71E0709F48EC20330FCE71F07C6
:1022600021F140F401153CE7130789F001301C47C8
:1022700011F13EC00B359CE7190739F10C35ECE73D
:102280001E07D9F00A351C4799F581E01FC00E944E
:1022900036282FEF34E38CE0215030408040E1F7C6
:1022A00000C000000E9452248FCE6FEF7FEF80E0CD
:1022B00090E00E948E2B0E94B40D8091BD0182FBA4
:1022C000882780F991E0892701C080E00E944817A3
:1022D0000FC00631FCE71F0709F45DC280914A0276
:1022E0008272F801E052F847E531F10508F469C25D
:1022F000F701828100811181882349F0C8010E9481
:102300007127D82E682FC8010E94C62704C0C801B3
:102310000E94AD27D82EB8018D2D0E94B6140E94C0
:10232000D614B82E192F982EF7010281A580A294F9
:102330009FE0A922809140028770B9F00023A9F0A4
:10234000812F807F803421F080E28B0D883068F00F
:102350008091BD0182FF09C082E00E942B1780910D
:1023600040028770DD24D3948111D12CC12EC294F8
:102370008FE0C8228C2D90E08C30910508F0DCC1F4
:10238000FC01EC56FF4F0C94E62B812F807F1F70D1
:10239000882311F01295107F0023B9F0112309F45E
:1023A000B4C180E28B0D883010F0911006C090917E
:1023B0004A02192B10934A0205C090914902192B29
:1023C000109349020E94EF16A0C18B2D0E945D2838
:1023D000112309F4B1C180E28B0D883088F1992076
:1023E00079F11095909149021923109349022BC05D
:1023F000812F807F1F70803211F01295107F8B2DFE
:10240000992029F0F1E09F1609F441C04FC0809156
:10241000BD0182FD1BC0002369F0112339F09091AA
:102420004A02192B10934A020E94EF1680E00E9484
:10243000902882C180E00E945D28112309F47CC1AC
:10244000812F0E94E8160E94EF1676C1002381F0CA
:1024500080914B02AA2051F021E0A21207C0182B54
:10246000181709F469C110934B0266C1812B16C07D
:10247000A11003C00E94E21635C031E0A31609F492
:102480005BC1812F0E944C280E94E21655C1002397
:1024900041F085E08A1508F44FC1812F0E9453282E
:1024A0004BC194E09A1508F447C11CC0002349F0C1
:1024B000AA2099F3F701858180FF27C18F7085835A
:1024C000ECCFAA2079F0893341F4FFEF27EE33E017
:1024D000F15020403040E1F72AC18FE39CE9019799
:1024E000F1F725C1812F0E944C2826C1812F8695A6
:1024F0008695837019F0813061F01EC1002321F0B0
:102500008B2D912F937002C080E090E00E942B25CC
:1025100019C1002321F08B2D912F937002C080E010
:1025200090E00E9406250EC1812F8370A9F501114C
:1025300007C14B2D429546954770440F440F8B2D94
:102540008F7090E09C01042E01C0220F0A94EAF7DC
:10255000B4FE08C08FE090E001C0880F4A95EAF70A
:10256000809501C080E0169516951370123069F0C1
:1025700088F490914C02113019F0822B892302C00B
:10258000922B892B0E94FC27DBC0822B90914C025E
:102590008927F8CF822BF6CF002319F0812F817085
:1025A00001C08695882309F4CBC04B2D42954695F2
:1025B0004770440F440F8B2D8F7090E09C01042EC8
:1025C00001C0220F0A94EAF7B4FE08C08FE090E041
:1025D00001C0880F4A95EAF7809501C080E0169502
:1025E00016951370123059F078F4909167021130FB
:1025F00019F0822B892309C0922B892B06C0822BCC
:1026000090916702892701C0822B0E94E02798C021
:102610001F70002339F0812F0E94F0278B2D0E941C
:1026200053288EC08B2D0E944C28812F0E94E327B7
:1026300087C08B2D92EF991681F1991538F0E0EF54
:102640009E1659F0F1EF9F1619F15BC023EF921619
:1026500059F134EF9316C1F054C0002381F084E0A7
:102660008A1508F469C01F7181E090E0012E01C055
:10267000880F0A94EAF790916702892720C095E0B5
:102680009A1508F459C0EFCF8091BD0182FD1AC0A0
:10269000002329F0812F8F7127C00023D9F3812FC8
:1026A0008F710E94E32748C0002341F01F7181E031
:1026B000012E01C0880F0A94EAF701C080E00E9451
:1026C000E0273AC0002399F01F71812F0E94F02764
:1026D0008091BD0182FF07C0E8E01E9FC001112468
:1026E000836080934002812F0E94F02725C081E003
:1026F0000E942B17F1E0FA15F8F482E00E942B17E4
:102700001BC0002321F0AA2029F28B2D90CEAA20F5
:1027100031F2893341F42FEF37EE83E0215030401E
:102720008040E1F704C0EFE3FCE93197F1F700C026
:1027300000008B2D0E945D2888EF8C0D843010F4F2
:102740000E945025DD2009F4B1C08091400280FD37
:10275000ADC0F70112828595859585950E94F02779
:10276000C7010E94670E80914002859585958595E9
:102770000E94E3279BC080914A028A7A91E009F483
:1027800090E09093FF0181111AC069E280E092E02D
:102790000E94EC2411C08091FF01811185C089E263
:1027A000E0E0F2E026E032E09281891301C012827B
:1027B00031962E173F07C1F70E94EF1605CC65E34F
:1027C000E5CFE056FF4F0C94E62B8091AE0480FFDE
:1027D00012C08E7F8093AE046091AE047091AF04FE
:1027E0008091B0049091B1040E94152910927A044E
:1027F0000E941C20E9CB81608093AE0461E0869545
:1028000050C043E659E26DE679E22CC04DE659E24C
:1028100063E679E227C04FE053E269E173E222C048
:1028200049E153E26FE073E21DC045EF52E262E01E
:1028300073E218C042E053E265EF72E213C04BED61
:1028400052E268EE72E20EC048EE52E26BED72E2C6
:1028500009C045E95FE167EA7FE104C047EA5FE15B
:1028600065E97FE10E941520AFCB61E081E019C0EE
:1028700065E082E011C068E086E00EC06EE089E0AD
:102880000BC064E18FE008C067E185E105C061E04D
:1028900088E107C062E289E10E94012095CB61E0F6
:1028A00083E20E94282990CB85E37ACF2D96E2E13E
:1028B0000C94382B80E008959091BC0192FF0DC0DC
:1028C000282F2871283019F4877F846006C0282FAC
:1028D0002471243011F48B7F886093FF0DC0282F62
:1028E0002871283119F4877E846106C0282F24714D
:1028F000243111F48B7E88612091BD0120FF0DC031
:10290000382F3871383019F4877F816006C0382F2E
:102910003171313011F48E7F886021FF0DC0282F76
:102920002871283119F4877E816106C0282F217112
:10293000213111F48E7E886194FD877E0895F8948C
:10294000E82FE295EF70F0E031A1282F2F7081E0A1
:1029500090E001C0880F2A95EAF7982F909593236D
:1029600091A392A1892B82A378940895462F672F73
:102970007A3038F44730B8F48430A8F40E94A9269D
:1029800008957D3F31F441110EC0843060F441E080
:1029900006C07C3F41F4411106C0843020F460E061
:1029A0000E940326089580E090E00895CF93DF937E
:1029B0008238910569F1B0F48133910509F477C04B
:1029C00048F48932910509F469C08A32910509F405
:1029D00073C092C08533910509F45BC089339105BA
:1029E000B9F08AC0833E910591F138F4803E91059B
:1029F000D1F0823E910531F17FC0863E9105D9F13B
:102A0000873E9105E9F1843E910509F075C028C023
:102A10002091BC0120FD5BC021FD59C02091BD016A
:102A200023FD61C069C08091BC0180FD4AC08091D6
:102A3000BD0180FF4CC08091BC0184FD50C183EE7C
:102A400090E04FC18091BC0182FF3EC0F4CF8091E5
:102A5000BC0182FD39C08091BD0180FD38C0EBCF43
:102A60008091BD0181FF39C08091BC0184FD37C1D7
:102A700087EE90E036C18091BC0183FF2BC0F4CF7C
:102A80008091BC0183FD26C08091BD0181FD25C0E0
:102A9000EBCF8091BC0185FD26C022C08091BC0196
:102AA00085FD1EC08091BD0183FF1DC00AC08091BD
:102AB000BC0186FD1BC01DC08091BC0186FD19C0F4
:102AC00015C089E390E00DC182EE90E00AC180EE6E
:102AD00090E007C186EE90E004C184EE90E001C171
:102AE00085E390E0FEC089E290E0FBC08AE290E0DE
:102AF000F8C081E390E0F5C0EC01811530E5930763
:102B000008F053C0811560E4960720F0CE019F7055
:102B1000906AE7C0803E910588F58D3C910518F0DC
:102B2000CE019065DEC0883A9105C0F4853A9105E2
:102B300050F08C2F855AC82FD0E0C95BDE4F8881BA
:102B400090E09064CEC08130910509F4C5C008F4CE
:102B5000C6C0049708F4C3C0CE01C3C0813C910530
:102B600008F0BDC08C2F885AC82FD0E0CC0FDD1FD5
:102B7000C65BDE4F888199819464B3C08115904211
:102B800058F08D2F8F710E945C14282F2F71CE0169
:102B900099279062922BA5C0C11581E0D807E0F675
:102BA000C83ED10508F09BC0D7CFC03692E5D90703
:102BB00008F053C0C03422E5D207B8F08C2F8F71D3
:102BC0008695869570E2879FA00111248C2F8370D3
:102BD00021E030E0B90102C0660F771F8A95E2F765
:102BE000CB019C68842B952B7CC0C03232E5D30787
:102BF00040F08C2F8F7190E0982F8827816F906A1A
:102C000070C0C11562E5D607B0F08C2F8695869509
:102C100020E2829FA00111248C2F837021E030E0FC
:102C2000B90102C0660F771F8A95E2F7CB01842BAA
:102C3000952B9D6856C08C2F8F710E945C1495E077
:102C4000D695C7959A95E1F7CF70D0E0DC2FCC27C9
:102C5000D0699E01282BC90144C0C03A72E5D7074C
:102C600008F58C2F8F71C03892E5D907A8F48695A6
:102C7000869570E2879F900111248C2F837041E02C
:102C800050E0BA0102C0660F771F8A95E2F7CB01C8
:102C90009A68822B932B25C090E0982F8827846F09
:102CA000906A1FC0C03C22E5D20750F48C2F8F7170
:102CB0000E945C148F7190E0982F8827906211C059
:102CC000C03E32E5D30758F4CE018F719927982F73
:102CD0008827806F906A05C081E090E002C080E0A4
:102CE00090E0DF91CF91089580E090E00E946A2B00
:102CF000873E9E4F19F40E94E81F089580E00895D2
:102D000067EE7EEF80E090E00E948E2B60E082E034
:102D100090E00E94702B60E083E090E00E94702BB6
:102D200010924C0260E074E184E090E00E948E2BEF
:102D300060E086E090E00E94702B6FEF87E090E00B
:102D40000E94702B40E050E0BA0188E090E00E94C1
:102D5000822B60E08DE090E00E94702B40E050E01C
:102D6000BA0188E190E00E94822B60E087E190E068
:102D70000E94702B40E050E0BA018CE190E00E948C
:102D8000822B60E070E080E290E00E948E2B40E0B9
:102D900050E0BA0188E190E00E94822B80E00E941E
:102DA000B91F0E94D81F40E050E0BA018FE090E0C8
:102DB0000E94822B40E050E0BA0183E190E00E9443
:102DC000822B089580914B02811110924B0208953D
:102DD000809590914A02892380934A0208959091A8
:102DE0004A0280914902982B9093000280914B02F5
:102DF000882389F0892B80930002E2E0F2E097E0DB
:102E000080E0915029F021912223D9F38F5FF9CFEF
:102E100081110E94E21648E050E061E472E080E037
:102E200092E00E94312C892BA9F088E0E0E0F2E0EA
:102E3000A1E4B2E001900D928A95E1F7E091BE0421
:102E4000F091BF04309731F00280F381E02D80E0F3
:102E500092E0099508952091400280958223809305
:102E60004002982F977099F430E0482F082E000CFC
:102E7000550B2417350759F09091BD0192FF07C0FB
:102E80008595859585950E94E327109240020895C7
:102E90009091BD0192FB222720F9281779F080FB41
:102EA00092F99093BD016091BC017091BD0184E0E5
:102EB00090E00E948E2B82E00E942B170895809153
:102EC0003F0290910E02891719F08F5F8770FBCF38
:102ED00008950F931F93CF93DF9380910D028295F6
:102EE0008F7009F05AC080910A02882309F455C0F6
:102EF00080913F0210910E026091080270910902C8
:102F0000C0910B02D0910C0291E06F3F09F090E06C
:102F1000292F06E0811709F440C0209721F07F3F58
:102F200021F030E003C031E001C0322F90E030FDED
:102F300031C0089FF001099FF00D1124DF01A15F4E
:102F4000BD4F11963C911197371324C03C91361315
:102F500021C012963C91129731111CC013964D91CD
:102F60005C9114974C1B5D0B483C510598F4809183
:102F70000D028F70806180930D02EC5EFD4F8081A9
:102F80008F708061808388E092E00E94670E0E94CB
:102F90005F1703C001968770BDCFDF91CF911F915E
:102FA0000F910895A1E1B0E0E8EDF7E10C94232B37
:102FB0008C0185E0F801DE011D9601900D928A9545
:102FC000E1F7F801E28090910802609109024091D6
:102FD0000B0250910C024115510531F06F3F31F455
:102FE00081E09F3F19F403C081E001C080E0F82F29
:102FF000F1709F2E80FD1BC1F80130812181C380BB
:10300000D48088E0A82E82E0B82EF0900A02F60163
:10301000E41BF50BFF2009F4C7C080910D02E83CCA
:10302000F10508F092C0482F407F09F051C06213AB
:1030300011C093130FC0FE2CE1100CC08F70806183
:1030400080930D02C5010E94670E80910D02F80168
:1030500085832AC1C114D10431F02F3F31F481E0BE
:103060003F3F19F403C081E001C080E080FD03C050
:1030700081E08E2502C080E090E0F82FF170FF2EF5
:1030800080FF1CC080913F0240910E0256E08417E1
:1030900009F4E8C090E0589FF001599FF00D112409
:1030A000E15FFD4F6181261306C06081631303C099
:1030B0006281E61203C001968770E9CFFE2CEE20F4
:1030C00009F4F2C080910D02816080930D0249C025
:1030D000621306C0931304C0E11002C0F80186C059
:1030E000C8010E94FF27882351F1EE2041F1209171
:1030F0000D02822F82958F7090E0029774F080917C
:1031000008029091090298878F831986DB86CA8608
:103110002C87CE0107960E94670E86E0F801A8E092
:10312000B2E001900D928A95E1F70E9469170AC0FA
:103130006217C9F0C8010E94FF2781111EC0C80193
:103140000E94670EFF24F394AFC0482F407F81F7A1
:1031500088E092E00E94670E86E0F50111928A9560
:10316000E9F7F12CA1C09313E5CFE110E3CFF8010B
:103170008583C8010E94670E54C0EE2001F32091A0
:103180000D02822F82958F7090E0029734F2809129
:103190000802909109029A8389831B82DD82CC8286
:1031A0002E83CE010196B7CFE83CF105D0F5FE2C79
:1031B000EE2029F2621327C0931325C020910D023F
:1031C00020FD18C0822F82958F70482F50E0411546
:1031D000510581F0F80125834F30510541F08F5F93
:1031E000982F9295907F822F8F70892B8583C801AD
:1031F0000E94670E86E0F801A8E0B2E001900D920F
:103200008A95E1F751C0C8010E94FF27811185CF3F
:1032100080910D02816080930D02C8010E94670EAB
:1032200043C086E0F50111928A95E9F73DC0EE2092
:1032300009F485CFC8010E94FF27F82E882309F4DE
:103240007ECF86E0F801A8E0B2E001900D928A9569
:10325000E1F780910802909109020E94A0270E9444
:10326000691722C03D872E878D859E850E94A027E5
:10327000292F22952F70223028F49F7039F0811168
:1032800005C00BC0243028F49F7049F4805E88305C
:1032900020F0C8010E94670E9F2CF92C05C0F80190
:1032A0009581907F99F7F9CF8F2D6196EBE00C9483
:1032B0003F2BAAE0B0E0EFE5F9E10C94232BAE013F
:1032C0004F5F5F4F7A018AE0FA0111928A95E9F720
:1032D0000EE111E06A01AA24A394B12CF8018081C7
:1032E0008F3F09F441C0F894E82FE295EF70F0E0C9
:1032F00021A18F70A50102C0440F551F8A95E2F7E6
:10330000CA01922F982B91A392A18095892382A321
:10331000789400C0E8E2F1E0912C31E021912F3F58
:1033200089F0A22FA295AF70B0E090968C9190E0BA
:103330002F7002C0959587952A95E2F780FD02C00F
:10334000832F01C080E0982A330F51E0EF32F50758
:1033500029F7F80180818F3F11F00E949F14F0EA55
:10336000FA95F1F7F60190820F5F1F4FFFEFCF1A2A
:10337000DF0A41E00832140709F0B0CF4AE050E01C
:10338000B70182EB91E00E94312C892B89F08AE011
:10339000F701A2EBB1E001900D928A95E1F781E08F
:1033A00080934F020E94B72490934E0280934D0267
:1033B00080914F02811102C080E020C080914D02B7
:1033C00090914E020E949C240597B0F34AE050E091
:1033D00062EB71E085EF91E00E94312C892B59F06E
:1033E0008AE0E2EBF1E0A5EFB1E001900D928A9561
:1033F000E1F781E001C080E010924F022A96EBE0F5
:103400000C943F2BCF93DF93C0917104D091720441
:103410008A30B1F420916802CE018B569240622F1F
:1034200070E00E94082B281B822F66E00E94A42BCC
:10343000C82FC15008F48FC080E20E94021AF9CF51
:103440008D30E9F4CB56D24020916802622F70E0B3
:10345000CE010E94082B281B822F9E01280F311DB0
:103460002115324018F080E0C0E0D0E0C80FD11D37
:10347000C559DD4FD0937204C09371046CC096E0BF
:10348000FE01ABE6B4E001900D929A95E1F7803E23
:1034900030F086E0FE0111928A95E9F70BC0F6E064
:1034A0008F9FB001112461547C4F46E050E0CE0163
:1034B0000E94532BC0917104D091720446E050E0F9
:1034C000BE018BE694E00E94312C892B49F19E01CC
:1034D0002B563240A90185E0569547958A95E1F72C
:1034E00081E090E0BC0102C0660F771F4A95E2F7C9
:1034F0004091690250916A02462B572B2B5F3F4F38
:1035000065E0369527956A95E1F702C0880F991F07
:103510002A95E2F7842B952B90936A028093690297
:103520009E012556324040916802642F70E0C90127
:103530000E94082B481B463010F4240F311D211522
:1035400082E0380710F020E030E025593D4F3093FD
:10355000720420937104DF91CF910895CF93DF938C
:10356000EC01FE018491882321F00E94021A219629
:10357000F8CFDF91CF91089590916802899FC001A3
:103580001124811522E0920714F080E090E0855923
:103590009D4F909372048093710408958091670207
:1035A000982F9670963011F4886001C0877F0E9432
:1035B000E0270895EF92FF920F931F93CF93DF932D
:1035C000EC017B0164E670E088E70E941A2A8C0116
:1035D000EC0EFD1ECE15DF0561F017FD0AC0FE01E1
:1035E000849164E670E00E948D2A8C012196892BDB
:1035F00089F30E94042BC801CDB7DEB7E6E00C9436
:10360000442BAAE2B0E0E7E0FBE10C942B2BEFE5C2
:10361000F2E087E692E02091F10021938E179F0758
:10362000D1F780916002833009F463C030F48130B7
:1036300071F0823009F49DC0B4C08A3009F489C0A9
:103640008B3009F46EC0893009F0ABC020C0809186
:103650005F02813A09F0A5C08091E800877F8093DE
:10366000E8008091630290916402892B21F468E064
:1036700083E592E003C060E080E090E070E00E94AB
:103680009B238091E8008B778093E8008AC080912B
:103690005F02813209F085C08091630290916402DB
:1036A000009719F0029709F07CC08091E800877FAD
:1036B0008093E8008091E80082FD05C080915D0262
:1036C0008111F8CF6EC02091F3008091F20090E05C
:1036D000922B029731F48091F100813011F0863005
:1036E00021F48091F100809352028091E8008B7761
:1036F00054C080915F02813A09F053C08091630207
:1037000090916402892B09F04CC08091E800877F7A
:103710008093E8008091E80080FFFCCF80910F014A
:1037200037C080915F028132E1F580916302909110
:103730006402892BB1F58091E800877F8093E800CF
:103740000E9447238091610280930F010E943628D6
:1037500028C080915F02813221F58091E800877F47
:103760008093E8000E944723809162028093510277
:1037700018C080915F02813AA1F48091E800877FB0
:103780008093E8008091E80080FFFCCF8091510297
:103790008093F1008091E8008E778093E8000E948A
:1037A00047238091E80083FFDFC180915F02909101
:1037B0006002492F50E04A30510508F0D5C1FA01A6
:1037C000EB54FF4F0C94E62B803821F0823809F03F
:1037D000CBC108C080915B0290915C02992389F073
:1037E00082600FC0809163028F70873008F0BCC187
:1037F0008093E9008091EB0085FB882780F9109287
:10380000E9009091E800977F9093E8008093F100A1
:103810001092F10070C1282F2D7F09F0A5C18823D7
:1038200019F0823061F0A0C180916102813009F00D
:103830009BC1933009F080E080935C022EC08091A0
:10384000610281112AC0809163028F702FEF280FCF
:10385000263008F089C18093E9002091EB0020FF19
:103860001CC0933021F48091EB00806214C09091D1
:10387000EB0090619093EB0021E030E0A90102C0E1
:10388000440F551F8A95E2F74093EA001092EA0030
:103890008091EB0088608093EB001092E9008091AA
:1038A000E800877F8093E8000E9447235DC1811173
:1038B0005BC1109161021F778091E3008078812BBA
:1038C0008093E3008091E800877F8093E8000E9466
:1038D00047238091E80080FFFCCF8091E30080685F
:1038E0008093E300111102C082E001C083E0809365
:1038F0005D023AC18058823008F036C120916102E1
:10390000309162022C3D53E0350779F583E08A83DC
:103910008AE289834FB7F894DE01139620E03EE0F7
:1039200051E2E32FF0E050935700E49120FF03C0F1
:10393000E295EF703F5FEF708E2F90E0EA3010F06D
:10394000C79601C0C0968D939D932F5F243149F790
:103950004FBF8091E800877F8093E8006AE270E0C3
:10396000CE0101960E949B23B4C080916302909186
:103970006402432F552743305105A9F068F44130C4
:10398000510509F400C14230510509F0EDC08BE545
:1039900090E0E4E2F3E04BC04132510529F14232BC
:1039A000510589F1E1C0C901992781309105A1F044
:1039B00058F0029709F0D8C0E1E9F3E0E4918E2FC6
:1039C00090E0E1E9F3E030C0EBEBF3E0E4918E2F1F
:1039D00090E0EBEBF3E028C0E5EAF3E0E4918E2F12
:1039E00090E0E5EAF3E020C08330910508F0BCC028
:1039F000880F991FFC01EB57FE4F0190F081E02DDD
:103A000089E090E014C08330910508F0ADC0FC015E
:103A1000EE0FFF1FE158FE4F0190F081E02DDC0119
:103A2000A458BE4F8C9190E0009709F49DC020915E
:103A3000E800277F2093E80020916502309166021C
:103A40002817390708F4C90140E0009789F120914F
:103A50005D02222309F43DC02530D9F12091E80010
:103A600023FD37C02091E80022FD2FC02091E800FF
:103A700020FFEBCF4091F3002091F20030E0342B97
:103A8000009759F02830310540F444914093F100FB
:103A9000319601972F5F3F4FF3CF41E0283031053A
:103AA00009F040E02091E8002E772093E800CDCF88
:103AB0004111CDCF0AC080915D02882351F085303D
:103AC00041F08091E80083FD04C08091E80082FF0E
:103AD000F2CF8091E8008B778093E80045C0803872
:103AE00009F042C08091E800877F8093E8008091D0
:103AF0005E028093F1008091E8008E77D3CE811131
:103B000033C080916102909162029927029764F517
:103B10008091E800877F8093E80010916102109304
:103B20005E020E944723111106C08091E30087FDC9
:103B300002C081E001C084E080935D0242E061EC5C
:103B400081E00E94662342E261EC84E00E946623E9
:103B500042E261EC82E00E94662342E260EC83E094
:103B60000E94662380915D028091E80083FF10C06F
:103B70008091E800877F8093E8008091EB0080626D
:103B80008093EB0005C082E190E0EFE7F3E04FCFD8
:103B9000AA96E3E00C94472B1F920F920FB60F9258
:103BA00011242F933F934F935F936F937F938F9342
:103BB0009F93AF93BF93CF93DF93EF93FF93C09106
:103BC000E900CF708091EC00D82FD17080FDD0E853
:103BD0001092E9008091F000877F8093F000789444
:103BE0000E94011B1092E9008091F0008860809390
:103BF000F000CD2BCF70C093E900FF91EF91DF91E2
:103C0000CF91BF91AF919F918F917F916F915F9174
:103C10004F913F912F910F900FBE0F901F901895CD
:103C2000E8EDF0E080818E7F80831092E2001092B8
:103C3000DA001092E100A0EEB0E08C9181608C93EC
:103C400080818F77808319BCA7EDB0E08C918E7F47
:103C50008C9380818F7E8083109250020895A0E023
:103C6000B0E0E5E3FEE10C94262BC8EDD0E08881BE
:103C70008F7E8883E7EDF0E080818160808384E03F
:103C800082BF81E08093500288818E7F888302EE1C
:103C900010E0F80110821092DA0081EEC82ED12CCB
:103CA000F601108288818F77888388818068888375
:103CB00088818F7D888319BC10925D0210925E020C
:103CC00010925C0210925B0290EEE92EF12CF7014B
:103CD00080818B7F808388818160888342E060E07F
:103CE00080E00E946623F60180818E7F8083F80148
:103CF000808181608083808188608083F7018081FA
:103D00008E7F8083888180618883CDB7DEB7E8E0CD
:103D10000C94422B1F920F920FB60F9211242F93E7
:103D20003F934F935F936F937F938F939F93AF9343
:103D3000BF93EF93FF938091E10082FF09C08091D0
:103D4000E20082FF05C08091E1008B7F8093E1005B
:103D50008091DA0080FF2AC08091D80080FF26C0C1
:103D60008091DA008E7F8093DA008091D90080FF05
:103D700018C080E189BD82E189BD09B400FEFDCF94
:103D800081E080935D028091500281110FC00E94FA
:103D9000101E0E942F1E8091E20084608093E2003A
:103DA00005C019BC10925D02109250028091E10092
:103DB00080FF17C08091E20080FF13C08091E20075
:103DC0008E7F8093E2008091E20080618093E20028
:103DD0008091D80080628093D80019BC85E08093E0
:103DE0005D028091E10084FF30C08091E20084FF99
:103DF0002CC080E189BD82E189BD09B400FEFDCF00
:103E00008091D8008F7D8093D8008091E1008F7ED3
:103E10008093E1008091E2008F7E8093E2008091A8
:103E2000E20081608093E20080915E02882311F0BD
:103E300084E007C08091E30087FD02C081E001C0FB
:103E400083E080935D0280915D028091E10083FFB9
:103E500027C08091E20083FF23C08091E100877F2B
:103E60008093E10082E080935D0210925E02809177
:103E7000E1008E7F8093E1008091E2008E7F80934D
